:1000000003C003C003C003C003C003C003C003C0D8
:100080001DC034C033C032C031C030C02FC02EC0FC
:100090002DC02CC02BC02AC029C028C027C026C014
:1000A00025C024C023C022C021C020C01FC01EC044
:1000B0001DC01CC01BC01AC019C018C00000000021
:1000C0000000000000000000000000000000000030
:1000D00000000000000000000000000011241FBE0E
:1000E000CFEFD2E0DEBFCDBF08D420C4C9CF009788
:1000F00009F40895E8EBFBE03197F1F70197F7CFAA
:10010000807F9B01205F3F4FDB01FC01E61BF70B6B
:10011000EA0FFB1F459154914D935D93A217B307CE
:10012000A1F70895FC01E07F93E090935700E895D4
:1001300007B600FCFDCF0895CF93DF939B01205FAE
:100140003F4FDB01FC01E61BF70BEA0FFB1FCD91D4
:10015000DD9141E00E0140935700E8951124A2176C
:10016000B30781F725E0FC0120935700E89507B617
:1001700000FCFDCFDF91CF910895CF93DF93CDB7F2
:10018000DEB760970FB6F894DEBF0FBECDBFBE01DD
:100190006F5F7F4F90E080E0B3DF8FEF9FEF9A8338
:1001A00089839C838B839E838D8398878F839A8793
:1001B00089879C878B879E878D87988B8F8790E018
:1001C00080E0B0DFBE016F5F7F4F90E080E0B4DF82
:1001D00060960FB6F894DEBF0FBECDBFDF91CF9112
:1001E0000895EF92FF920F931F93CF93DF93CDB7B4
:1001F000DEB760970FB6F894DEBF0FBECDBF10E03C
:1002000000E045E00A3E14076CF060960FB6F894E3
:10021000DEBF0FBECDBFDF91CF911F910F91FF9039
:10022000EF90089530E020E0F801E05FFC4FE20F2E
:10023000F31FC9018E7F48E0EA3FF407ECF44591D3
:10024000549161E070E06C0F7D1F860F971FFC01D9
:10025000518340832E5F3F4F2031310529F77801CC
:10026000F6EEFF1AC7015EDFBE016F5F7F4FC70169
:1002700063DF005F1F4FC5CF41E050E04C0F5D1FB3
:10028000840F951F4FEF5FEFE2CFCF93DF93CDB792
:10029000DEB760970FB6F894DEBF0FBECDBF8FEF0D
:1002A0009CEC9A8389839C838B839E838D83988720
:1002B0008F839A8789879C878B879E878D87988B6A
:1002C0008F8790E080E02EDFBE016F5F7F4F90E070
:1002D00080E032DF60960FB6F894DEBF0FBECDBF70
:1002E000DF91CF910895CF9387B3836087BBC19887
:1002F000CAEF81E090E0FBDEC19A81E090E0F7DE9A
:10030000C198C150B1F7CF910895F0E0E0E00994B1
:1003100016C019FA10859315000009021200010198
:1003200000803209040000000000000012011001EA
:10033000FF000008D0165307060200000001112438
:100340001FBECFEFD2E0CDBFDEBF21E0A0E0B1E025
:1003500001C01D92AC32B207E1F780C1DC018FEF22
:100360009FEF332715C02D912827722F229527271D
:10037000822F269526952827239522703217779568
:100380002795822F8927972F76952795972782275C
:10039000615048F7809590958D939D930895CF93E4
:1003A000CFB7CF93C395B09BE9F7B09B09C0B09B83
:1003B00007C0B09B05C0B09B03C0B09B01C0A7C0E5
:1003C000DF93C0910E01DD27CA5EDE4FB09B02C0F5
:1003D000DF91EBCF2F930F931F9306B32FEF00FB0B
:1003E00020F94F933F9316B34FEF012700FB21F9FC
:1003F0003BE031C04E7F012F16B3216028C0102F83
:100400004D7F2260000006B329C04B7F2460012F7E
:10041000000016B32BC016B3477F28602AC04F7E5A
:1004200006B320612CC04F7D16B320622FC04F7BD6
:1004300006B3206432C0422706B349934FEF000051
:10044000102710FB20F916B31370C9F1297F91F220
:10045000012700FB21F906B3237F89F2315058F1BF
:10046000102710FB22F916B3277E79F2012700FB33
:1004700023F92F7C81F206B3102710FB24F92F7982
:1004800071F200C016B3012700FB25F92F7359F252
:1004900000C006B3102710FB26F9223040F200C03E
:1004A00016B3012700FB27F9243028F64F77206880
:1004B00016B30000F9CF10E21ABF00271DC03B5051
:1004C0003195C31BD04010E21ABF0881033C19F1DB
:1004D0000B3409F120910C011981110F1213EDCF8A
:1004E000093641F10D3211F0013E39F7CAE01AB771
:1004F00015FD02C0CA95D9F7009314013F914F91A1
:100500001F910F912F91DF91CAB7C5FD4BCFCF91AE
:10051000CFBFCF91089520911401222379F3109138
:1005200012011123E1F43430E2F0309312012093F0
:100530000D0117C00091120101308CF40AE53091D1
:100540000F0134FD10C000930F01C1E0D1E00FC0D6
:100550002795A8F45150A9F4220F0000F9CF4AE5DD
:1005600003C042ED01C0432FC4E1D0E032E017B335
:100570001360C09A17BB08B320E413E05F93012710
:1005800056E008BB279520F4515021F4220FF9CFF3
:10059000012756E000003B5A08BBD0F2279528F40B
:1005A000515029F4220F0000F9CF012756E027957A
:1005B00008BB20F4515021F4220FF9CF012756E057
:1005C0002991332308BB21F60C7F10911301110FE1
:1005D000C651D04008BB11F010930C0110E21ABFB5
:1005E000016017B31C7F402F4C7F5F9100C000C09B
:1005F00008BB17BB48BB82CFB09BFECF09D008D049
:1006000001D000D0975A70917400791B70937400D8
:100610006FEF8BE29927669576B370298B9671FB05
:1006200067F906B200FE6623B1F70895F20130972C
:1006300091F02AEF421629E1520619F480917400D4
:1006400090E021E00C0120935700E8951124CF01A0
:1006500002962C0108958FEF9CECF3CFEAEFF9E1BD
:10066000E491EF3F19F0E0937400000088ED80936F
:10067000710087E081BDB89A88EB9BE0ECE2F1E085
:100680003197F1F70197D1F7B8988AE580930F0178
:100690008FEF8093000180B5826080BD8BB7806250
:1006A0008BBFC298712C312C512C412CC0EADFE059
:1006B00014E686B3837009F014E6115029F4109201
:1006C000130110920C0198DF0AB605FEA1C067DE87
:1006D00080E28ABFA89522E032120CC0E0E0FAE185
:1006E000E054F10983E080935700E8953097C1F713
:1006F000512C412C832D803409F08EC0F2013297A9
:10070000E1158AE1F80720F485E080935700E89529
:10071000312C80911201835087FD2BC090910D01E7
:100720009D3229F5883019F583EC809301018AE523
:1007300080930F0180911701807690911801882392
:1007400009F49EC0712C911175C082E09AE19093DA
:1007500011018093100188E090911E01911105C054
:1007600090911D01981708F4892F80930001109231
:10077000120180910F0184FF30C0809100018F3FF2
:1007800061F1C82F893008F0C8E0982F9C1B909326
:1007900000019091010128E892279093010188239C
:1007A00081F0E0911001F0911101A2E0B1E08C2FF5
:1007B00094919D9331968150D9F7F0931101E09374
:1007C00010016C2F82E091E0C9DDCC5FCC3019F0D4
:1007D0008FEF80930001C0930F01C30101963C018C
:1007E000803B24E0920729F4EDEFF9E1E491EF3F3B
:1007F000C9F48C7409F47FC0BA980AB605FE56CFC6
:1008000085E1B09B85E18150E1F780E28ABF4ECF60
:10081000219709F04ECF5ECF843009F079CFCD2BF0
:1008200009F077CFBA98B8981BBE10BC84B783BBC9
:1008300014BE6CCD913079F44114510411F480E070
:100840008BCF80911B01807F482E50901C0181E14D
:1008500087BFE895F4CF933081F48091190190918E
:100860001A01E4DE80911B0190911C01DFDE842DD2
:100870008F7029F790E4392E6FCF9F73392EDFCF19
:100880002091190110920A0191110AC010920B01D6
:100890002AE031E082E030931101209310015CCF17
:1008A000953029F4209313012AE031E0F4CF9630FB
:1008B00091F480911A01813041F48CE19AE1909396
:1008C00011018093100182E147CF823009F0B7CF48
:1008D0008AE09AE1F4CF983051F0993019F42093DE
:1008E0001501E2CF81E09A30F9F280E0DDCF25E119
:1008F00031E081E0D0CFBA9A80CF88B318BA87B3FD
:100900008FEF87BB8AEF90E0F2DB87B317BA8AEFED
:1009100090E0EDDBF89431DC64DCB7DCE4DC8DEFF7
:1009200099E100DCF2DC90E080E00895F894FFCFDC
:040000030000008079
:00000001FF
